:0400000086EF25F072
:08000800046ED8CF05F0E0CF33
:1000100006F00001E9CF0CF0EACF07F0E1CF08F0DD
:10002000E2CF09F0D9CF0AF0DACF0BF0F3CF12F01C
:10003000F4CF13F0FACF14F0F5CF15F0F6CF16F099
:10004000F7CF17F000C00EF001C00FF002C010F0A3
:1000500003C011F09DAA30EF00F09EBAEBEF03F061
:10006000CEEF03F00EC000F00FC001F010C002F0A0
:1000700011C003F00CC0E9FF07C0EAFF078E08C0FB
:10008000E1FF09C0E2FF0AC0D9FF0BC0DAFF12C0CE
:10009000F3FF13C0F4FF14C0FAFF15C0F5FF16C03C
:1000A000F6FF17C0F7FF045006C0E0FF05C0D8FFF9
:1000B0001000F76AC20FF66E000EF7220900F55025
:1000C0001200000000000000005F000000070007B1
:1000D00000147F147F14242A7F2A122313086462D9
:1000E00036495522500005030000001C2241000043
:1000F00041221C0014083E081408083E080800505D
:10010000300000080808080800606000002010089F
:1001100004023E5149453E00427F40004261514940
:10012000462141454B311814127F1027454545396A
:100130003C4A4949300171090503364949493606A7
:100140004949291E003636000000563600000814C2
:100150002241001414141414004122140802015105
:100160000906324979413E7E1111117E7F49494984
:10017000363E414141227F4141221C7F494949414C
:100180007F090909013E4149497A7F0808087F0033
:10019000417F41002040413F017F081422417F40C0
:1001A0004040407F020C027F7F0408107F3E4141A7
:1001B000413EF76AC20FF66E010EF7220900F550B4
:1001C00012007F090909063E4151215E7F09192964
:1001D00046464949493101017F01013F4040403FC6
:1001E0001F2040201F3F4038403F6314081463071E
:1001F000087008076151494543007F4141000204EE
:100200000810200041417F000402010204404040E8
:100210004040000102040020545454787F48444474
:10022000383844444420384444487F38545454189F
:10023000087E0901020C5252523E7F0804047800E5
:10024000447D40002040443D007F10284400004190
:100250007F40007C041804787C0804047838444407
:1002600044387C14141408081414187C7C08040402
:10027000084854545420043F4440203C4040207CD3
:100280001C2040201C3C4030403C44281028440C9A
:100290005050503C4464544C440008364100000027
:1002A0007F00000041360800100808100878464119
:1002B0004678F76AC20FF66E020EF7220900F55073
:1002C00012001E216121123C4140217C38545655B8
:1002D0001820555555782055545578205556547842
:1002E00020545554781C2262221038555555183820
:1002F00055545518385455561800457C4100004552
:100300007D410000457E400078151415787814155D
:1003100014787C5456554424547854487E097E49B8
:1003200049384545453838454445383845464438C8
:100330003C4141217C3C4142207C0C5150513C3895
:10034000454445383C4140413C0000000000204805
:100350003E49620000000000000000000040683ECE
:100360000902205456557800447E410038444645E1
:10037000383C4042217C7C090505787C0911217CB0
:100380007E2525261800F76A960FF66E030EF722D3
:100390000900F55012002D2D2D2D2D2D2D2D000095
:1003A000F76AB00FF66E030EF7220900F55012003F
:1003B000202020202020202020202020202020203D
:1003C000202020202020202020202020202020202D
:1003D00020202020202020202000F76AEA0FF66E3F
:1003E000030EF7220900F5501200202020202020C3
:1003F00020202020202020202020202020202020FD
:100400002000F76A120FF66E040EF7220900F5506D
:1004100012004D6F6E00F76A260FF66E040EF7227B
:100420000900F550120054756500F76A3A0FF66E30
:10043000040EF7220900F550120057656400F76AB0
:100440004E0FF66E040EF7220900F55012005468A4
:100450007500F76A620FF66E040EF7220900F55078
:10046000120046726900F76A760FF66E040EF722E4
:100470000900F550120053617400F76A8A0FF66E96
:10048000040EF7220900F550120053756E00F76A4A
:100490009E0FF66E040EF7220900F55012004A6115
:1004A0006E00F76AB20FF66E040EF7220900F550DF
:1004B000120046656200F76AC60FF66E040EF72258
:1004C0000900F55012004D617200F76ADA0FF66EFE
:1004D000040EF7220900F550120041707200F76A0D
:1004E000EE0FF66E040EF7220900F55012004D6172
:1004F0007900F76A020FF66E050EF7220900F55033
:1005000012004A756E00F76A160FF66E050EF72296
:100510000900F55012004A756C00F76A2A0FF66E52
:10052000050EF7220900F550120041756700F76AC1
:100530003E0FF66E050EF7220900F55012005365C6
:100540007000F76A520FF66E050EF7220900F5509B
:1005500012004F637400F76A660FF66E050EF722FD
:100560000900F55012004E6F7600F76A7A0FF66EAA
:10057000050EF7220900F550120044656300F76A82
:100580008E0FF66E050EF7220900F5501200746DFD
:100590006300F76AA20FF66E050EF7220900F55008
:1005A000120074646E00F76AB60FF66E050EF7223D
:1005B0000900F550120074757000F76ACA0FF66EE4
:1005C000050EF7220900F550120067657400F76AFE
:1005D000DE0FF66E050EF7220900F5501200736566
:1005E0007400F76AF20FF66E050EF7220900F55057
:1005F000120073617600F76A060FF66E060EF72298
:100600000900F550120072647300F76A1A0FF66E53
:10061000060EF7220900F550120072657300F76AA2
:100620002E0FF66E060EF7220900F550120000009C
:10063000202A2A736920706F7765722075702A2AC4
:100640002000202121200000202A2A7369207475AF
:100650006E652A2A2000737400006D6F0000202A46
:100660002A73692074756E652A2A200020202020B4
:10067000202020202020200043545F4D4A443A206F
:10068000256C750A0D00544D433A2043433D2578AF
:10069000204C544E3D2578200A0D0000544D433A1D
:1006A000205349443D2578200A0D0000544D433A1B
:1006B00020543D257520463D25752044503D257527
:1006C0002000443D2575206469723D2575204558FC
:1006D000543D257520004556543D254C75204C4F02
:1006E000433D254C750A0D000A0D00004652455148
:1006F0003A2025332E31670A0D00544154503A20D8
:10070000746D630A0D00544154503A2054410A0D4F
:100710000000544154503A2054500A0D00005441F6
:1007200054503A202D0A0D0050533A2025730A0DDB
:10073000000050493A20254C780A0D005254613A85
:100740002025730A0D005254623A2025730A0D00C9
:100750000900F5520DE0F6CFA5F3F7CFA6F3F5505B
:100760009EA8FED7AD6EA5C3F6FFA6C3F7FFF0D7D0
:10077000000C030EEA6EA60EE96EEF500EE0140EAA
:10078000016E006A002EFED7012EFBD7BF0E006E51
:10079000002EFED700D0EF2EF2D7000CC20EF66E60
:1007A000070EF76ED5DF040E0301A56FFA0EA66FD4
:1007B0000001DFDF0301A52FF9D7FF00000132EFB1
:1007C00000F044656661756C7420696E74657272C0
:1007D0007570740D0A00036A56507E0FE96E000EA4
:1007E0000320EA6E9EAAFED7AECFEFFF56C0A5F358
:1007F000010E56241F0B566E5750565C02E1A5C3DE
:1008000056F09E9A32EF00F00A0D0A0D00000A0A17
:100810000D20303836202D20464D20524453202DB7
:10082000204D6F62696C652054756E6572204D6F46
:1008300064756C65202A2A20746563686465736931
:10084000676E2E62650A0D2000007A6F6E653D208E
:1008500025750A0D00007A6F6E653D2025750A0D1D
:1008600000007A6F6E653D2025750000464D2052D0
:1008700044532000544120005450200020202000E8
:10088000202A2A656E7465722A2A2000202A2A707E
:1008900072657365742073617665642A2A2000008E
:1008A000736176656400202A2A72696768742A2A4F
:1008B0002000202A2A6C6566742A2A200000202A3B
:1008C0002A75702A2A200000202A2A646F776E2A4F
:1008D0002A200000465245513A2025332E31670A1E
:1008E0000D200000202A2A707265736574207361E0
:1008F0007665642A2A200000202A2A20676F746FF8
:1009000020707265736574202575202A2A200000E6
:100910002046524551353D2573200000202A2A20CB
:100920007361766520707265736574202575202A61
:100930002A2000000900F6CF81F3F7CF82F3F550AB
:100940009EA8FED7AD6E81C3F6FF82C3F7FF0301F9
:10095000802F01D002D00001EDD70001000C03016F
:100960008351016A825D03E282C300F00CD0006A09
:10097000080E846F823700368351005CD8B0006E59
:100980000136842FF7D70001000C015080C382F399
:10099000640E0301836F0001E2DF00C080F30150A9
:1009A000300E08E1030181A30ED081B70CD081B9CC
:1009B000200E04D003018197819981810126015085
:1009C0009EA8FED7AD6E80C382F30A0E836F00012E
:1009D000C6DF00C080F30150300E08E1030181B78B
:1009E0000BD081A109D081B9200E00010126015050
:1009F0009EA8FED7AD6E0301300E802780519EA8C1
:100A0000FED7AD6E0001000C080E0301A36FA353C7
:100A100011E08A9C939C00D0A2BF03D08A9E939E33
:100A200002D08A8E939E00D08A8C939CD890A23755
:100A3000A307EDD70001000C8B9494948B929492B1
:100A400094C3A2F3E1DF8B849494000C196AF2BE84
:100A5000198EF29E640E0301A66F00018ADE19BE94
:100A6000F28E898E929E8B8494948A8C939C8B9028
:100A70009490196AF2BE198EF29E0A0E0301A66FB7
:100A8000000177DE19BEF28E8B809490196AF2BE57
:100A9000198EF29E010E0301A66F00016ADE19BED7
:100AA000F28EAE0E0301946F0001C6DFA00E0301AB
:100AB000946F0001C1DF730E0301946F0001BCDF6E
:100AC000A10E0301946F0001B7DF0301946B0001D5
:100AD000B3DFA20E0301946F0001AEDF0301946B3C
:100AE0000001AADFA40E0301946F0001A5DFA80E88
:100AF0000301946F0001A0DF3F0E0301946F00011A
:100B00009BDFAD0E0301946F000196DF8E0E030193
:100B1000946F000191DFB00E0301946F00018CDF30
:100B20000B0E0301946F000187DFB10E0301946F78
:100B3000000182DF310E0301946F00017DDFB30EEF
:100B40000301946F000178DFF00E0301946F000140
:100B500073DF8A0E0301946F00016EDF640E0301E0
:100B6000946F000169DF8B0E0301946F000164DF55
:100B7000780E0301946F00015FDF8C0E0301946F08
:100B800000015ADF640E0301946F000155DFBB0EB4
:100B90000301946F000150DF3E0E0301946F0001CA
:100BA0004BDFBE0E0301946F000146DF3E0E0301D2
:100BB000946F000141DF870E0301946F00013CDF59
:100BC000ACC094F339DF810E0301946F000134DF70
:100BD000ADC094F331DF820E0301946F00012CDF6E
:100BE000ADC094F329DF830E0301946F000124DF6D
:100BF000ADC094F321DFAF0E0301946F00011CDF41
:100C0000B2EF26F08B9494948B829492A0C3A2F3BB
:100C1000FBDEA1C3A2F3F8DE8B849494000CAE0E2D
:100C20000301946F000108DF150E0301946F0001AA
:100C300003DF0301946B0001FFDE5F0E0301946F7D
:100C40000001FADE750E0301946F0001F5DE030169
:100C5000946B0001F1DE3F0E0301946F0001ECDEA6
:100C60000301346B336B335303E13451180809E04B
:100C7000A06BA16B0001C6DF0301332BD8B4342B6A
:100C8000F2D7AF0E946F0001D7DEB4EF26F0150E49
:100C90000301946F0001D0DE84C394F3CDDE5F0EB8
:100CA0000301946F0001C8DE750E0301946F00010B
:100CB000C3DE85C394F3C0DE3F0E0301946F0001D1
:100CC000BBDEB56B84C3B4F0B76B85C3B6F0000C64
:100CD000B051C70804E1800EB06F03D102D1B0510A
:100CE000FC0804E1810EB06FFCD0FBD0B051E908E4
:100CF00004E1820EB06FF5D0F4D0B051E20804E107
:100D0000830EB06FEED0EDD0B051E40804E1840E54
:100D1000B06FE7D0E6D0B051E00804E1850EB06FC7
:100D2000E0D0DFD0B051E50804E1860EB06FD9D035
:100D3000D8D0B051E70804E1870EB06FD2D0D1D03F
:100D4000B051EA0804E1880EB06FCBD0CAD0B051E0
:100D5000EB0804E1890EB06FC4D0C3D0B051E808ED
:100D600004E18A0EB06FBDD0BCD0B051EF0804E1F1
:100D70008B0EB06FB6D0B5D0B051EE0804E18C0E3A
:100D8000B06FAFD0AED0B051EC0804E18D0EB06FB3
:100D9000A8D0A7D0B051C40804E18E0EB06FA1D086
:100DA000A0D0B051C50804E18F0EB06F9AD099D091
:100DB000B051C90804E1900EB06F93D092D0B051F9
:100DC000E60804E1910EB06F8CD08BD0B051C6080C
:100DD00004E1920EB06F85D084D0B051F40804E1E4
:100DE000930EB06F7ED07DD0B051F60804E1940E22
:100DF000B06F77D076D0B051F20804E1950EB06FA5
:100E000070D06FD0B051FB0804E1960EB06F69D07E
:100E100068D0B051F90804E1970EB06F62D061D08C
:100E2000B051D60804E1990EB06F5BD05AD0B051E2
:100E3000DC0804E19A0EB06F54D053D0B051F808DA
:100E400004E19B0EB06F4DD04CD0B051A30804E12B
:100E50009C0EB06F46D045D0B051D80804E19D0E2D
:100E6000B06F3FD03ED0B051D70804E19E0EB06FB6
:100E700038D037D0B051830804E19F0EB06F31D025
:100E800030D0B051E10804E1A00EB06F2AD029D0D3
:100E9000B051ED0804E1A10EB06F23D022D0B051C3
:100EA000F30804E1A20EB06F1CD01BD0B051FA08B9
:100EB00004E1A30EB06F15D014D0B051F10804E1D5
:100EC000A40EB06F0ED00DD0B051D10804E1A50E24
:100ED000B06F07D006D0B051DF0803E1A60EB06FA7
:100EE00000D09BEF07F003019B35A06FA037A03720
:100EF000F80EA0179C31006E003200321F0E001653
:100F00000050A0119E6F9C39006E0036E00E001656
:100F100000509D119F6F9EC3A0F39FC3A1F30001DA
:100F200071DE000CB0511F0802E32CD104D0B05187
:100F30007F0801E2CDD6B051A60801E223D1B16B02
:100F4000B1510408D8A0CCD0B0514F080CE3B05137
:100F5000E00F050DF3CFB2F0B151B225036A59ECA1
:100F600000F0B36F1DD0B0517F080CE3B051B00F4B
:100F7000050DF3CFB2F0B151B225036AD9EC00F000
:100F8000B36F0ED0B051A6080BE3B051800F050D22
:100F9000F3CFB2F0B151B225036A59EC01F0B36F4F
:100FA0000301936B0001BC510301935DD8B495D04C
:100FB000926B92510808D8B48ED09B6B0001BB5144
:100FC0000F0B03019C6F9C31966F9B31956F96338D
:100FD00095339633953396339533963395339633CD
:100FE0009533030E96170001BA51F00B03019B6F66
:100FF0009C6B9C31986F9B31976F983397333F0E62
:1010000098170001BA510F0B03019B6F9C6B9B3526
:10101000996F9C359A6F99379A37FC0E9917B3C020
:1010200000F09251016E04E0D8900032012EFCD7FE
:1010300000A03DD09B6B0001B9510F0B03019C6FC9
:101040009C339B339C339B339C339B339C339B332C
:101050009C339B339C339B33030E9C179B25956FCE
:10106000000E9C21966F0001B851F00B03019B6F9D
:101070009C6B9C339B339C339B333F0E9C17030E1E
:101080009B25976F000E9C21986F0001B8510F0BA4
:1010900003019B6F9C6B9B379C379B379C37FC0EE7
:1010A0009B17030E9B25996F000E9C219A6F946BE2
:1010B0000001BD510301945D0BE095C39BF397C301
:1010C0009CF399C39DF300010EDF0301942BF0D72D
:1010D000010E92276ED7932B65D70001B12B30D725
:1010E00003019B6B0001BB510F0B03019C6F9C31F3
:1010F000966F9B31956F9633953396339533963330
:1011000095339633953396339533030E9617000136
:10111000BA51F00B03019B6F9C6B9C31986F9B3114
:10112000976F983397333F0E98170001BA510F0B02
:1011300003019B6F9C6B9B35996F9C359A6F993718
:101140009A37FC0E9917936B0001BC510301935D14
:1011500019E0926B9251080813E0946B0001BD51A5
:101160000301945D0BE095C39BF397C39CF399C374
:101170009DF30001B8DE0301942BF0D7922BEAD740
:10118000932BE2D70001FAEF08F0150E0301946FDC
:10119000000152DCB4C094F34FDCBC51060DF35097
:1011A000B4250301926F000E0001B5210301936F76
:1011B00092C394F3000140DC750E0301946F0001AB
:1011C0003BDCB6C094F338DCBD51080DF350B625B6
:1011D0000301926F000E0001B7210301936F010E0E
:1011E000925F000E935B92C394F3000125DC91C3E0
:1011F000B0F098D6BC51060DF350B427000EB523BD
:10120000000C0900F6CF34F3F7CF35F3F5CF91F3A7
:10121000BCDF34C3F6FF35C3F7FF0301332F01D022
:1012200002D00001EED70001CEEF26F0015037C307
:1012300082F3640E0301836F0001AFEC04F000C081
:1012400037F30150300E08E1030138A30FD038B74F
:101250000DD038B9200E04D0030138973899388161
:10126000012601C091F3000190DF030137C382F32F
:101270000A0E836F0001AFEC04F000C037F3015099
:10128000300E08E1030138B70AD038A108D038B9C8
:10129000200E0001012601C091F377DF0301300E1B
:1012A000372737C391F3000170DF000C0900F552B6
:1012B0000CE0F6CF84F3F7CF85F3F5CF91F365DF3C
:1012C00084C3F6FF85C3F7FFF1D7000C070E0301B7
:1012D000906F903D01D01AD08FC300F09051016EF5
:1012E00004E0D8900032012EFCD700B002D08B98D9
:1012F00001D08B88949800008B96949600008B8682
:10130000949600008B9694969007E3D70001000C0A
:10131000800E946E050E006E002EFED78B9694966E
:101320008B9894980000899A929A0000480E0301C5
:101330008F6F0001CBDF87C38FF3C8DF88C38FF3C4
:10134000C5DF89C38FF3C2DF8AC38FF3BFDF8BC3CF
:101350008FF3BCDF8CC38FF3B9DF8DC38FF3B6DFA0
:101360008EC38FF3B3DF0000898A929A000C0301C9
:10137000876B070E886F883D01D018D08B969496A6
:1013800000008B869496948882A80BD0010E006E84
:101390008851016E04E0D8900036012EFCD7005031
:1013A000871300008B9694968807E5D787C301F0D2
:1013B0000001000C0301846B800E946E00008B967C
:1013C00094968B989498899A929A0000800E8F6FC9
:1013D00000017CDF0000900E946E0000C8DF01C0A9
:1013E00084F30000898A929A800E946E030184C36C
:1013F00001F00001000C8E0E006E85C301F084C365
:1014000002F0036A015209E102C001F0026A080E0B
:10141000005E015202E1006A08D0D89001BE04D0FB
:10142000023601360006F9D7019E000C03019151E6
:10143000D8B471D0006E9551D8B46DD0002604E3B5
:10144000810E002668E204D07F0E005E64E363E054
:1014500092C399F39651991B928F968F945198034A
:10146000F4CF9BF393519703F4CF03F0F3CF9AF3A8
:101470009803F3509B27F4509A23000E03229451B3
:101480009703F3509B27F4509A23000E026A03221D
:10149000022292519803F3509A27F4500322000E2F
:1014A000022292519703F3500326F4500222000EB9
:1014B000016A012294519603F3509A27F4500322B3
:1014C000000E0222012293519603F3500326F4509A
:1014D0000222000E012292519603F3500226F4508C
:1014E0000122002A01BE05D09A37033602360136A2
:1014F0000006000E9AAF0AD0032A022201220150F0
:1015000005E1025003E1035001E1002A99BF018E79
:1015100099AF019E04D0006A016A026A036A000161
:10152000000C800ED8A202D00301961B03019B6B16
:101530009C6B92C39AF396519A1B9151D8B4DFD009
:10154000996F006E9551D8B4E3D0995FD8B483D029
:101550003EE396C39FF39F8F97C39EF398C39DF37B
:101560009C6BD8909F339E339D339C33992FF8D733
:101570009AAF03D09B81E0D09B9199919B89030EF8
:10158000EA6E940EE96EEBD09B999ABF0AD099A1AE
:1015900013D09F339E339D339C33002AD8B4C7D0D9
:1015A0000BD09FBF0CD0D8909C379D379E379F376C
:1015B0000006D8B4BCD0F5D79B8D6DD09B9D92C34F
:1015C0009AF392AF02D09F8FABD09F9FA9D095C3C3
:1015D00099F395C300F09151995F92C39FF39F8F48
:1015E00093C39EF394C39DF39C6BD8909F339E331B
:1015F0009D339C33992FF8D79AAF03D09B839CD00F
:101600009B9399919B8B030EEA6E980EE96EA7D07F
:101610009B9B9ABF0AD099A113D09F339E339D33D1
:101620009C33002AD8B483D00BD09FBF0CD0D89065
:101630009C379D379E379F370006D8B478D0F5D7B2
:101640009B8F29D09B9F96C39AF396AF02D09F8F12
:1016500067D09F9F65D096C39FF39F8F97C39EF3DC
:1016600098C39DF39AAF04D09F9F9B8565D09B95AF
:101670009C6B9991030EEA6E940EE96E70D09ABF3E
:101680001CD092C39AF399A106D09F339E339D3309
:101690009C33002A4CE09CAF0BD09D2B09E19E2B84
:1016A00007E19F2B05E19F339E339D33002A3FE0E6
:1016B0009BBD84D79BBFC6D71CD0800E9F1B9FAFFE
:1016C00004D03AD096C39AF30AD092C39AF39F53A8
:1016D00006E19E5304E19D5302E1006A21D09FBFC1
:1016E00008D0D8909C379D379E379F37002EF7D76C
:1016F0001ED09AAF02D09F8F13D09F9F11D095C359
:1017000000F096C39FF397C39EF398C39DF308D050
:1017100091C300F092C39FF393C39EF394C39DF3D0
:101720009FC301F09EC302F09DC303F034D0006A52
:10173000016A026A036A2FD09C6B9D1F9E1F9F1F28
:101740009C1F9C2B05E19D2B03E19E2B01E19F2B10
:101750009BB112D79BB354D79BB589D7B3D7EF5062
:101760009D2705E39E2B03E19F2BD8B49981ED5271
:10177000EF509E2703E39F2BD8B49981ED52EF5091
:10178000EFBE01D0800A9F27D8B099819BB9FCD6C3
:101790009BBB3ED774D70001000C03018851D8B41D
:1017A000A5D0946F8C51D8B4A1D0945F05E37F0E7F
:1017B0009427D8B09BD006D0810E945FD8A096D045
:1017C000D8B494D094C300F0016A026A036A936BA0
:1017D00089C392F3928F8AC391F38BC390F3190E4E
:1017E000946F8F51905F0DE2010E915F0AE2925F5C
:1017F00008E2935F06E2932B922B912B8F51902757
:1018000028D08E51915F12E2010E925F0FE2935F3A
:101810000DE2932B922B8E5191278F51902719E334
:10182000912B17E1922B15E1932B13D08D51800949
:10183000925F0EE2010E935F0BE2932B8D518009B4
:1018400092278E519127E9E3922BE7E1932BE5D77D
:101850000380942F01D00BD0D890903791379237D6
:101860009337D8900336023601369537BAD795A10B
:1018700006D0D890013202320332953302D00006EE
:1018800035E095BF1ED0D890903791379237933777
:101890008F51905F07E2010E915F04E2925F02E2D6
:1018A000935F1AE38E51915F05E2010E925F02E2AF
:1018B000935F12E38D518009925F03E2010E935F03
:1018C0000BE3032A09E1022A07E1012A05E1002AC4
:1018D0000DE001320232033289C394F38D51941B1F
:1018E00094AF02D0018E06D0019E04D0006A016A36
:1018F000026A036A0001000CEF5210E0EACF7AF3AB
:10190000E9CF79F3EF509EA8FED7AD6E7AC3EAFF18
:1019100079C3E9FFE92AD8B4EA2AEED7000C8E0E83
:10192000006E03018351005E84C302F085C301F0A1
:10193000028E005209E0D890025202E1015204E006
:1019400002320132002EF7D784AF05D0011E021EED
:10195000012AD8B4022A0001000C5E0EF66E060EB3
:10196000F76E196AF2BE198EF29EA8EC03F019BE4A
:10197000F28E7CC394F37BC393F37AC392F379C35F
:1019800091F30301986B976B480E966F850E956FD8
:1019900000014CDD03C080F302C07FF301C07EF381
:1019A00000C07DF380C386F37FC385F37EC384F3D9
:1019B0007DC383F3B4DF02C082F301C081F303016E
:1019C00082511D0804E30BE18151AF0808E2825106
:1019D000290806E2FF0A03E18151300801E221D023
:1019E00082C383F3846B846B81C385F3866B200E83
:1019F000876F886B82C389F381C38AF38B6B8C6B8F
:101A00008D6B8E6B000184DCD5DC01C083F3000E8E
:101A1000030101BE010E000A04E100000001F4D739
:101A200003010001000C010EA16FF80EF66E080E06
:101A3000F76E100E0301806F00019AEC04F0A1C054
:101A400080F31B0E0301816F0001C5EC04F00A0E48
:101A5000F66E090EF76E040E0301806F00019AEC1A
:101A600004F0A151100DF3CF33F30301F2CF3AF399
:101A7000F29EAA6A33C3A9FFA69CA69EA680A85080
:101A80003ABFF28E346F010E33253A6FF2CF3BF33B
:101A9000F29EAA6A3AC3A9FFA69CA69EA680A85059
:101AA0003BBFF28E356F856B34C384F30001A3DC3A
:101AB00003C039F302C038F301C037F300C036F376
:101AC00039C394F338C393F337C392F336C391F316
:101AD0000301986B976B966B870E956F0001A6DCE0
:101AE00003C039F302C038F301C037F300C036F346
:101AF0000301856B35C384F300017DDCD89239C3C3
:101B000094F338C393F337C392F336C391F303C00E
:101B100098F302C097F301C096F300C095F301DD7E
:101B200003C039F302C038F301C037F300C036F305
:101B300039C38BF338C38AF337C389F336C388F3C9
:101B400003018F6B8E6B480E8D6F850E8C6F0001BD
:101B500024DE03C039F302C038F301C037F300C0FC
:101B600036F3100EF66E090EF76E070E0301806F46
:101B700000019AEC04F037C3EAFF36C3E9FFBCDE8C
:101B8000200E9EA8FED7AD6E39C37CF338C37BF31D
:101B900037C37AF336C379F3E0DE51EF0FF089985B
:101BA0009298899A929A800E946E090E936E8B96F3
:101BB00094968B9894988A829392196AF2BE198EA1
:101BC000F29E0A0E0301A66F0001B9EC03F019BEE4
:101BD000F28E89989298196AF2BE198EF29E0A0EB8
:101BE0000301A66F0001B9EC03F019BEF28E8988DB
:101BF0009298196AF2BE198EF29E0A0E0301A66F20
:101C00000001B9EC03F019BEF28E8A9293920B0E8A
:101C1000936E196AF2BE198EF29E0A0E0301A66F28
:101C20000001B9EC03F019BEF28E300EF66E060E0E
:101C3000F76E196AF2BE198EF29EA8EC03F019BE77
:101C4000F28E010E0301876F100E886F050E896FEB
:101C50008A6B8B6B8C6B8D6B8E6B000188EC09F043
:101C6000DAEC09F001C033F3000E030101BE010EEE
:101C7000000A18E1196AF2BE198EF29E640EA66F70
:101C80000001B9EC03F019BEF28E200E9EA8FED71B
:101C9000AD6E2A0E9EA8FED7AD6E200E9EA8FED772
:101CA000AD6EDED70001DAEC09F0013C19D0196AFB
:101CB000F2BE198EF29E640E0301A66F0001B9EC0C
:101CC00003F019BEF28E420EF66E060EF76E196A1A
:101CD000F2BE198EF29EA8EC03F019BEF28EE3D785
:101CE000A02D10D0120E0301876F886B110E896F23
:101CF0008A6B8B6B020E8C6F8D6B8E6B000188EC88
:101D000009F00FD0120E0301876F886B110E896FD7
:101D10008A6B8B6B010E8C6F8D6B8E6B000188EC68
:101D200009F0DAEC09F001C033F3000E030101BE43
:101D3000010E000A03E100000001F3D70001A051E9
:101D4000030810E1120E0301876F886B140E896F70
:101D50008A6B8B6B8C6B1D0E8D6F900E8E6F0001DE
:101D600088EC09F0DAEC09F001C033F3000E03014E
:101D700001BE010E000A04E100000001F3D70301D7
:101D8000120E876F886B150E896F8A6B8B6B010E35
:101D90008C6F8D6B8E6B000188EC09F0DAEC09F02A
:101DA00001C033F3000E030101BE010E000A04E17D
:101DB00000000001F3D70301120E876F886B150E28
:101DC000896F010E8A6F8B6B8C6F8D6B8E6B000130
:101DD00088EC09F0DAEC09F001C033F3000E0301DE
:101DE00001BE010E000A04E100000001F3D7030167
:101DF000120E876F886B150E896F020E8A6F550E53
:101E00008B6F010E8C6F8D6B8E6B000188EC09F06F
:101E1000DAEC09F001C033F3000E030101BE010E3C
:101E2000000A03E100000001F3D73F0E0001BF6F7D
:101E3000120E0301876F886B400E896F8A6B8B6B64
:101E4000BFC08CF38D6B8E6B000188EC09F0DAEC6F
:101E500009F001C033F3000E030101BE010E000AB8
:101E600004E100000001F3D70301480EF66E060EF0
:101E7000F76E196AF2BE198EF29E0001A8EC03F00B
:101E800019BEF28EDAEC09F001C033F3000E030143
:101E900001BE010E000A03E100000001F3D70001BA
:101EA000C2D5F2EF26F00301846B800E946E8B9600
:101EB00094968B989498899A929A0000C00E8F6F8E
:101EC000000166EC09F00000900E946E0000B7EC83
:101ED00009F001C084F3010E0301856F85511008DC
:101EE00011E00001B7EC09F001C086F3036A0301B9
:101EF0008551C00FE96E000E0320EA6E86C3EFFF26
:101F0000852BECD70000898A929A800E946E84C348
:101F100001F00001000C010E0301845F0CE3030ECD
:101F2000EA6E840EE96EEF5006E0040E006E002E9D
:101F3000FED7EF2EFAD700017CEF11F0016A026A9A
:101F4000006A036A0301875102E1865118E0100E0E
:101F5000886FD89084378537003603368751035C05
:101F600002E18651005C07E38651005ED8A00306BB
:101F70008751035ED88001360236882FEAD70001E8
:101F8000D7EF11F0030184518603F3CF01F0F4CFB2
:101F900000F08703F350002685518603F35000209C
:101FA000026E0001000C03019151B608916F036AA3
:101FB00092C395F3928FD890923393339433033234
:101FC000023201320032912FF6D795AF0BD0001EAE
:101FD000011E021E031E002AD8B4012AD8B4022A08
:101FE000D8B4032A0001000CD8B204D0030EEA6E64
:101FF000990EE96E006A016A026A036A0301996B2D
:102000009A6B9B6B9C6B98519711961195112CE0D4
:10201000200E9D6FD8909137923793379437993728
:102020009A379B379C3798519C5D08E197519B5D8F
:1020300005E196519A5D02E19551995D0FE3955145
:10204000995F9651D8A0963D9A5F9751D8A0973D39
:102050009B5F9851D8A0983D9C5FD8800036013690
:10206000023603369D2FD6D799C3EFFF9AC3ECFFF4
:102070009BC3ECFF9CC3ECFF0001000CE950030183
:10208000896F88518B6F1CE087C394F386C393F3E9
:1020900085C392F384C391F3986B976B200E966F70
:1020A000820E956F000116EC0AF003C087F302C0A0
:1020B00086F301C085F300C084F303018B2FE4D7BE
:1020C0007E0E006E016A85BF018E026A036AD89295
:1020D00087C394F386C393F385C392F384C391F3C8
:1020E00003C098F302C097F301C096F3956F000107
:1020F00091EC0AF003C087F302C086F301C085F3B8
:1021000000C084F387C394F386C393F385C392F32B
:1021100084C391F348DF03C087F302C086F301C094
:1021200085F300C084F3030187AF0DD08907898B45
:10213000841F851F861F871F842BD8B4852BD8B496
:10214000862BD8B4872B3B0E906F9A0E8F6FCA0EDA
:102150008E6F8D6B0A0E8B6F8851D8B4892BD88205
:10216000030EEA6E840EE96E87C394F386C393F37D
:1021700085C392F384C391F390C398F38FC397F30D
:102180008EC396F38DC395F300012EDF01500052EC
:1021900013E1030188298B5DD8A402D000010CD083
:1021A00089510DE00F0B8B5D01E044E289BF42D005
:1021B00089BD05D0200E37D0200E0301891789ABC9
:1021C0000FD0899B8851D8A489070050896F2D0EA4
:1021D000916F0001C5EC08F003018951006E896B15
:1021E00088518B5D0DE10050896F2E0E916F0001BB
:1021F000C5EC08F003018951006E200E8917000E0E
:10220000300E89AB10D0899B8851D8A48907005023
:10221000896F2D0E916F0001C5EC08F00301895103
:10222000006E896B300E002600C091F30001C5ECF2
:1022300008F00301D89290C394F38FC393F38EC335
:1022400092F38DC391F3986B976B966B0A0E956F13
:102250000001CADE03C090F302C08FF301C08EF309
:1022600000C08DF303018B2F7AD7000107EF12F026
:102270000301816B836B826B0001DAEC09F001C012
:1022800084F3000E030101BE010E000A02E100000A
:10229000F3D7140E876F886B896B8A6B8B6B8C6B93
:1022A0008D6B8E6B000188EC09F0DAEC09F001C04F
:1022B00084F3000E030101BE010E000A04E10000D8
:1022C0000001F3D70301220E876F886B896B8A6B3D
:1022D0008B6B8C6B8D6B8E6B000188EC09F0E3DDF2
:1022E00001C084F3000E030184BF010E000A05E162
:1022F000640E846F00010FD6F2D70001D56BC2C007
:10230000D4F0D4C0D5F0D46BC351D427000ED5235C
:10231000D5C085F3D4C084F3FBEC09F000C084F38E
:1023200001C085F302C086F303C087F3D89203C0CF
:1023300094F302C093F301C092F300C091F30A0E2C
:102340000301986FD70E976F230E966F780E956FD7
:10235000000191EC0AF000C084F301C085F302C0D3
:1023600086F303C087F303C08BF302C08AF301C076
:1023700089F300C088F303018F6B8E6B480E8D6F5D
:10238000850E8C6F0001CDEC0BF003C023F002C072
:1023900022F001C021F000C020F0D5C085F3D4C0E8
:1023A00084F30301876B640E866F0001C7D502C0FA
:1023B000D7F001C0D6F0D7C085F3D6C084F30301AF
:1023C000876B640E866F0001DDDD0150D45DD86F30
:1023D0000250D559D96F0301846B100E856F00012F
:1023E00047EC06F0BB6BBA6B0F0EB96FFF0EB86F00
:1023F000020EE96E23C087F322C086F321C085F365
:1024000020C084F3010E0301886F000137D6200E2F
:102410000301916F0001C5EC08F0D5C0DBF0D4C01A
:10242000DAF0230E0301876F886B896B8A6B8B6BE5
:102430008C6B8D6B8E6B000188EC09F034DD01C074
:1024400084F3000E030101BE010E000A03E1000047
:102450000001F4D70001C3AF03D0010E0301816F67
:10246000540E0301846F100E856F000147EC06F0D7
:10247000BB6BBA6B0F0EB96FFF0EB86F0301812DE6
:1024800009D0560EF66E060EF76E000156EC09F0F6
:1024900008D003015A0EF66E060EF76E000156ECD8
:1024A00009F0000C03017951080DF3CF7BF3846B25
:1024B0007BC385F3000147EC06F003017A6B7A5188
:1024C000100808E0200E916F0001C5EC08F0030130
:1024D0007A2BF5D70001000CF26BF06BF16BEA6A16
:1024E000F60EE96E000EC3EC01F00A000900F5508B
:1024F000EE6E0009FBE103012A6B0001EA6BE96B58
:10250000010EEA6EE96E000ED0EC01F00A0009003F
:10251000F550EE6E0009FBE1020EEA6E050EE96E63
:10252000000EEDEC01F00A000900F550EE6E000916
:10253000FBE1020EEA6E410EE96E000EEDEC01F0D9
:102540000A000900F550EE6E0009FBE1020EEA6E8A
:102550007D0EE96E000EEDEC01F00A000900F55069
:10256000EE6E0009FBE1020EEA6EB90EE96E000E96
:10257000EDEC01F00A000900F550EE6E0009FBE1F8
:10258000010EEA6E830EE96E000ED0EC01F00A0037
:102590000900F550EE6E0009FBE1020EEA6E230E13
:1025A000E96E000EEDEC01F00A000900F550EE6E48
:1025B0000009FBE1020EEA6E5F0EE96E000EEDEC23
:1025C00001F00A000900F550EE6E0009FBE1020E71
:1025D000EA6E9B0EE96E000EEDEC01F00A000900B8
:1025E000F550EE6E0009FBE1020EEA6ED70EE96EC1
:1025F000000EEDEC01F00A000900F550EE6E000946
:10260000FBE1240E0301876F020E886F896B8A6BD2
:102610008B6B8C6B8D6B8E6B000188EC09F0E86B1B
:102620000201FC6BFB6BFE6BFD6BF66BF56BF86BE5
:10263000F76B372C01D02CD00301796B000132DF0E
:10264000010E0301796F00012DDF1E0E0301846F5F
:10265000100E856F000147EC06F06C0EF66E060E4C
:10266000F76E56EC09F0040E0301796F00011ADFD2
:10267000050E0301796F000115DF060E0301796F66
:10268000000110DF070E0301796F00010BDF02016B
:102690000001000C5750565CFDE0036A57507E0F56
:1026A000E96E000E0320EA6EEFCF79F30301010E0D
:1026B00057241F0B576E79C301F00001D0EF17F0BC
:1026C0007AC303F0030179C3E9FF7AC3EAFFEF524B
:1026D00039E07AC37EF379C37DF37CC380F37BC397
:1026E0007FF380C303F07FC3E9FF80C3EAFFEF52AB
:1026F00016E07DC3E9FF7EC3EAFFEFCF81F380C31D
:1027000003F07FC3E9FF80C3EAFFEF50815D07E17B
:102710007D2BD8B47E2B7F2BD8B4802BE2D780C3FF
:1027200003F07FC3E9FF80C3EAFFEF5205E179C3FD
:1027300001F07AC302F009D0792BD8B47A2B0001CA
:10274000BFD70301000E016E026E000165EF18F0A5
:102750007AC37CF379C37BF37CC303F003017BC3AF
:10276000E9FF7CC3EAFFEF5206E07B2BD8B47C2B59
:102770000001F2D7030179517B5D006E7A517C59DB
:10278000036E00C001F00001000C03017D5302E163
:102790007E5342E079C3E9FF7AC3EAFFEFCF7FF3CC
:1027A0007CC303F07BC3E9FF7CC3EAFFEF507F5D8E
:1027B00017E07AC303F079C3E9FF7AC3EAFFEFCFEA
:1027C0007FF37CC303F07BC3E9FF7CC3EAFFEF50D8
:1027D0007F5D02E2FF0E01D0010E016E1FD00BD013
:1027E0007AC303F079C3E9FF7AC3EAFFEF5203E14A
:1027F000000E016E13D07AC303F07951792BD8B44F
:102800007A2B7CC303F07B517B2BD8B47C2B7D517E
:10281000D8B47E077D07BAD7000E016E0001000C08
:10282000E95003017E6F7D51806F1CE07CC394F3FF
:102830007BC393F37AC392F379C391F3986B976B4D
:10284000200E966F820E956F000116EC0AF003C001
:102850007CF302C07BF301C07AF300C079F303017B
:10286000802FE4D77E0E006E016A7ABF018E026A65
:10287000036AD8927CC394F37BC393F37AC392F335
:1028800079C391F303C098F302C097F301C096F3A4
:10289000956F000191EC0AF003C07CF302C07BF35A
:1028A00001C07AF300C079F37CC394F37BC393F344
:1028B0007AC392F379C391F3D3EC0FF003C07CF3A6
:1028C00002C07BF301C07AF300C079F303017CAF4F
:1028D0000DD07E077E8B791F7A1F7B1F7C1F792B83
:1028E000D8B47A2BD8B47B2BD8B47C2B3B0E856F15
:1028F0009A0E846FCA0E836F826B0A0E806F7D51B1
:10290000D8B47E2BD882030EEA6E790EE96E7CC3B2
:1029100094F37BC393F37AC392F379C391F385C3A2
:1029200098F384C397F383C396F382C395F30001AE
:10293000F4EC0FF00150005213E103017D29805D9A
:10294000D8A402D000010CD07E510DE00F0B805DA9
:1029500001E03CE27EBF3AD07EBD05D0200E31D0F2
:10296000200E03017E177EAB0DD07E9B7D51D8A437
:102970007E0700507E6F2D0E9EA8FED7AD6E7E5155
:10298000006E7E6B7D51805D0BE100507E6F2E0EE0
:102990009EA8FED7AD6E7E51006E200E7E17000EF3
:1029A000300E7EAB0ED07E9B7D51D8A47E070050AA
:1029B0007E6F2D0E9EA8FED7AD6E7E51006E7E6B93
:1029C000300E002600509EA8FED7AD6ED89285C36B
:1029D00094F384C393F383C392F382C391F3986B0C
:1029E000976B966B0A0E956F0001F4EC0FF003C025
:1029F00085F302C084F301C083F300C082F30301B6
:102A0000802F80D70001000C7BC381F37AC380F351
:102A100003017E5302E17F5327E07DC303F07CC3B3
:102A2000E9FF7DC3EAFFEF521FE081C303F080514D
:102A3000802BD8B4812B826F03C083F37DC303F056
:102A40007C517C2BD8B47D2BE96E03C0EAFFEFCF1D
:102A500084F383C3EAFF82C3E9FF84C3EFFF7E519F
:102A6000D8B47F077E07D5D77E5302E17F530FE0AE
:102A700081C303F08051802BD8B4812BE96E03C051
:102A8000EAFFEF6A7E51D8B47F077E07EDD77AC39D
:102A900001F07BC302F00001000C010EA16F1C0EBF
:102AA000F66E090EF76E100E0301806F00019AECAE
:102AB00004F0A1C080F31B0E0301816F0001C5EC7F
:102AC00004F02E0EF66E090EF76E040E0301806FF1
:102AD00000019AEC04F023C094F322C093F321C0C8
:102AE00092F320C091F30301986B976B480E966F99
:102AF000850E956F000116EC0AF003C07FF302C04B
:102B00007EF301C07DF300C07CF37FC38BF37EC3F3
:102B10008AF37DC389F37CC388F303018F6B8E6BCB
:102B20008D6B870E8C6F0001CDEC0BF003C086F32C
:102B300002C085F301C084F300C083F38FEC0CF076
:102B400001C07AF30301856B7AC384F3010E876FAA
:102B5000866B0001C2EC0FF002C085F301C084F364
:102B60000001FBEC09F0D8827FC394F37EC393F39A
:102B70007DC392F37CC391F303C098F302C097F333
:102B800001C096F300C095F391EC0AF003C086F300
:102B900002C085F301C084F300C083F38FEC0CF016
:102BA00001C07BF3A151100DF3CF79F30301AA6AA1
:102BB00079C3A9FF7AC3A8FFA69CA69EA684F2505B
:102BC000006EF29E0F01550EA76EAA0EA76EA6828A
:102BD000A6B2FED7A6940050F212010E0301792589
:102BE000806FAA6A80C3A9FF7BC3A8FFA69CA69E8C
:102BF000A684F250006EF29E0F01550EA76EAA0E2B
:102C0000A76EA682A6B2FED7A6940050F2120001CB
:102C100038EC11F0000C03017ABF10D00F0E006EDB
:102C2000793900160A0E005C03E2300E002602D04D
:102C30007A51002600509EA8FED7AD6E0F0E791770
:102C40000A0E795D02E2300E02D07A9F7A5179271E
:102C500079519EA8FED7AD6E0001000CE95003012A
:102C60007D6F3B0E846F9A0E836FCA0E826F816BED
:102C70000A0E7F6FD882030EEA6E790EE96E7CC36E
:102C800094F37BC393F37AC392F379C391F384C330
:102C900098F383C397F382C396F381C395F300013E
:102CA000F4EC0FF00150005213E103017F51010ACF
:102CB000D8A402D000010CD07D510CE00F0B7F5D39
:102CC00001E00EE27DBF0CD07DBD04D0200E03D00C
:102CD00003017D6B300E002600509EA8FED7AD6E1E
:102CE000D89284C394F383C393F382C392F381C3D2
:102CF00091F3986B976B966B0A0E956F0001F4EC4D
:102D00000FF003C084F302C083F301C082F300C05C
:102D100081F303017F2FAED70001000CE80EF66EA1
:102D2000060EF76E196AF2BE198EF29EA8EC03F039
:102D300019BEF28EEC0EF66E060EF76E060E03014D
:102D4000806F00019AEC04F0020EE96E23C07CF360
:102D500022C07BF321C07AF320C079F3010E030176
:102D60007D6F00015DDD0A0E9EA8FED7AD6E0D0ED3
:102D70009EA8FED7AD6EF22D0DD0FA0EF66E060EA1
:102D8000F76E196AF2BE198EF29EA8EC03F019BE16
:102D9000F28E2AD0F02D1CD0F12D0DD0060EF66E3D
:102DA000070EF76E196AF2BE198EF29EA8EC03F0B8
:102DB00019BEF28E0CD0120EF66E070EF76E196A5F
:102DC000F2BE198EF29EA8EC03F019BEF28E0CD062
:102DD0001E0EF66E070EF76E196AF2BE198EF29E7F
:102DE000A8EC03F019BEF28E280EF66E070EF76EF1
:102DF000040E0301806F00019AEC04F0EA6AF60EFB
:102E0000E96E7CEC0CF00A0E9EA8FED7AD6E0D0E9E
:102E10009EA8FED7AD6E320EF66E070EF76E040E4C
:102E20000301806F00019AEC04F0EAC079F3570EB9
:102E300003017A6F0001EFDEE9C079F3570E030159
:102E40007A6F0001E8DE0A0E9EA8FED7AD6E0D0E69
:102E50009EA8FED7AD6E03010D530BE10C5309E1A3
:102E60000B510608D8B06BD0FF0A03E10A51D9080C
:102E700066E20D5364E10C5362E10B5107085FE316
:102E800003E10A51EE085BE3430E9EA8FED7AD6E48
:102E9000540E9EA8FED7AD6E3D0E9EA8FED7AD6E19
:102EA00027C380F3110E816F0001C5EC04F03A0EC8
:102EB0009EA8FED7AD6E28C380F3010E0301816F7B
:102EC0000001C5EC04F0200E9EA8FED7AD6E030EE7
:102ED000EA6E2B0EE96E7CEC0CF0200E9EA8FED75D
:102EE000AD6E030EEA6E2F0EE96E7CEC0CF0200E38
:102EF0009EA8FED7AD6E16C380F3110E0301816F3D
:102F00000001C5EC04F02C0E9EA8FED7AD6E200E7D
:102F10009EA8FED7AD6E040EE96E0DC37CF30CC304
:102F20007BF30BC37AF30AC379F398DE0A0E9EA8EB
:102F3000FED7AD6E0D0E9EA8FED7AD6E03013C0E02
:102F4000F66E070EF76E050E806F00019AEC04F026
:102F5000010EEA6EE96E7CEC0CF00A0E9EA8FED71C
:102F6000AD6E0D0E9EA8FED7AD6E460EF66E070E28
:102F7000F76E050E0301806F00019AEC04F0010E5C
:102F8000EA6E830EE96E7CEC0CF00A0E9EA8FED76A
:102F9000AD6E0D0E9EA8FED7AD6E000C4AEF13F07D
:102FA00001C033F3030133510D080BE1036A000143
:102FB0007851580FE96E000E0320EA6EEF6A12D0C6
:102FC0000301036A00017851580FE96E000E0320D7
:102FD000EA6E33C3EFFF7851210802E2786B01D02B
:102FE000782B85D2030EEA6E490EE96E000EC9EC0D
:102FF00002F00A000900F550EE6E0009FBE1030E35
:10300000EA6E4E0EE96E000ED3EC02F00A000900E3
:10301000F550EE6E0009FBE1030EEA6E530EE96E09
:10302000000EDDEC02F00A000900F550EE6E00091A
:10303000FBE1030EEA6E580EE96E000EE7EC02F0BB
:103040000A000900F550EE6E0009FBE1030EEA6E7E
:10305000660EE96E000EF1EC02F00A000900F55070
:10306000EE6E0009FBE1030EEA6E6B0EE96E000ED8
:10307000FBEC02F00A000900F550EE6E0009FBE1DE
:10308000030EEA6E700EE96E000EBFEC02F00A004D
:103090000900F550EE6E0009FBE1030EEA6E750EB5
:1030A000E96E000E05EC03F00A000900F550EE6E23
:1030B0000009FBE103017A6B580E796F030E7C6FF8
:1030C000580E7B6F000160EF13F001C05DF3030148
:1030D0007A6B580E796F0001A8EC13F001500208CA
:1030E000D8B0F8D103017A6B580E796F030E7C6F5C
:1030F000490E7B6F7E6B030E7D6F0001C5EC13F0F4
:1031000001C048F303017A6B580E796F030E7C6F90
:103110004E0E7B6F7E6B030E7D6F0001C5EC13F0CE
:1031200001C04DF303017A6B580E796F030E7C6F6B
:10313000530E7B6F7E6B030E7D6F0001C5EC13F0A9
:1031400001C052F303017A6B580E796F030E7C6F46
:10315000580E7B6F7E6B030E7D6F0001C5EC13F084
:1031600001C057F303017A6B580E796F030E7C6F21
:10317000660E7B6F7E6B030E7D6F0001C5EC13F056
:1031800001C065F303017A6B580E796F030E7C6FF3
:103190006B0E7B6F7E6B030E7D6F0001C5EC13F031
:1031A00001C06AF303017A6B580E796F030E7C6FCE
:1031B000700E7B6F7E6B030E7D6F0001C5EC13F00C
:1031C00001C06FF303017A6B580E796F030E7C6FA9
:1031D000750E7B6F7E6B030E7D6F0001C5EC13F0E7
:1031E00001C074F3030148531BE1210E876F040EE5
:1031F000886F896B8A6B8B6B8C6B8D6B8E6B000110
:1032000088EC09F038EC11F06CEC12F038EC11F0AD
:10321000A66BA56B0B0EA46FB80EA36F5BD1030159
:103220004D531BE1210E876F0C0E886F896B8A6BE3
:103230008B6B8C6B8D6B8E6B000188EC09F038EC1E
:1032400011F06CEC12F038EC11F0A66BA56B0B0EC4
:10325000A46FB80EA36F3ED10301525327E1D40EE1
:10326000F66E080EF76E060E806F00019AEC04F001
:10327000020EE96E23C07CF322C07BF321C07AF3F7
:1032800020C079F3010E03017D6F000110EC14F0F2
:103290000A0E9EA8FED7AD6E0D0E9EA8FED7AD6E8F
:1032A000200E9EA8FED7AD6E15D103015753D8A4AA
:1032B000F1D0030E5D25796F030E7B6F5E0E7A6F82
:1032C0007D6B79C37CF37F6B050E7E6F000104EC90
:1032D00015F003015E510F0B856B846F0001FBEC51
:1032E00009F003C037F302C036F301C035F300C064
:1032F00034F303015F510F0B856B846F0001FBEC0E
:1033000009F003C03BF302C03AF301C039F300C037
:1033100038F3030160510F0B856B846F0001FBECE8
:1033200009F003C03FF302C03EF301C03DF300C00B
:103330003CF3030162510F0B856B846F0001FBECC2
:1033400009F003C043F302C042F301C041F300C0DF
:1033500040F337C394F336C393F335C392F334C3C6
:1033600091F30301986B976B480E966F850E956FDE
:10337000000116EC0AF000C079F301C07AF302C034
:103380007BF303C07CF33BC394F33AC393F339C399
:1033900092F338C391F30301986B976B200E966FED
:1033A000820E956F000116EC0AF0D8927CC394F35C
:1033B0007BC393F37AC392F379C391F303C098F379
:1033C00002C097F301C096F300C095F391EC0AF0A8
:1033D00000C079F301C07AF302C07BF303C07CF331
:1033E000D89203C094F302C093F301C092F300C0DB
:1033F00091F33FC398F33EC397F33DC396F33CC3A9
:1034000095F391EC0AF000C079F301C07AF302C0A1
:103410007BF303C07CF343C394F342C393F341C3F0
:1034200092F340C391F3CD0E0301986FCC0E976FCA
:103430004C0E966F7B0E956F000116EC0AF0D89239
:103440007CC394F37BC393F37AC392F379C391F370
:1034500003C098F302C097F301C096F300C095F340
:1034600091EC0AF003C047F302C046F301C045F3F4
:1034700000C044F347C37CF346C37BF345C37AF3F0
:1034800044C379F3ADEC0CF06CEC12F038EC11F0B5
:1034900021D00301655311E100014DEC15F0E40E5C
:1034A000F66E080EF76E196AF2BE198EF29EA8EC3F
:1034B00003F019BEF28E0ED003016A5304E100013D
:1034C0002DDC08D003016F5301E103D0745301E1F7
:1034D000FF000001EA6A580EE96E000E0FEC03F0DF
:1034E0000A000900F550EE6E0009FBE1786B07EF6A
:1034F00027F0030EEA6E360EE96EEF500EE0050E71
:10350000016E006A002EFED7012EFBD72E0E006E34
:10351000002EFED700D0EF2EF2D7000C928480A4AC
:103520006FD00301346B800EF66E080EF76E196AC9
:10353000F2BE198EF29E0001A8EC03F019BEF28EC5
:10354000928480A40ED00301342B050E366F000147
:10355000D0DF03013451630802E2000102D0000110
:10356000EFD7200E9EA8FED7AD6E2A0E9EA8FED7DE
:10357000AD6E34C380F31B0E0301816F0001C5ECF7
:1035800004F02A0E9EA8FED7AD6E200E9EA8FED790
:10359000AD6E3750020833E1030134516308D8B0EF
:1035A00002D000012CD000014DEC15F08C0EF66E0F
:1035B000080EF76E196AF2BE198EF29EA8EC03F09F
:1035C00019BEF28E0301846B856B000147EC06F097
:1035D0000F0EBB6FF00EBA6FB96BB86BA00EF66E24
:1035E000080EF76E56EC09F0020E0301356FFA0E65
:1035F000366F00017EDF0301352FF9D70001D0D0EF
:10360000928080A02AD0A60EF66E080EF76E196A78
:10361000F2BE198EF29EA8EC03F019BEF28E37505E
:1036200002081AE1210E0301876F0C0E886F896B67
:103630008A6B8B6B8C6B8D6B8E6B000188EC09F049
:1036400038EC11F06CEC12F038EC11F0A66BA56BB5
:103650000B0EA46FB80EA36FA3D083AC2AD0B20E0A
:10366000F66E080EF76E196AF2BE198EF29EA8EC7D
:1036700003F019BEF28E375002081AE1210E030141
:10368000876F040E886F896B8A6B8B6B8C6B8D6B6D
:103690008E6B000188EC09F038EC11F06CEC12F044
:1036A00038EC11F0A66BA56B0B0EA46FB80EA36FD0
:1036B00077D0928280A23BD0BE0EF66E080EF76ED7
:1036C000196AF2BE198EF29EA8EC03F019BEF28EB2
:1036D000375002082BE1928280A228D0BF2BBF5125
:1036E0003E0802E23F0EBF6F120E0301876F886B28
:1036F000400E896F8A6B8B6BBFC08CF38D6B8E6BAA
:10370000000188EC09F0DAEC09F001C035F3000E95
:10371000030101BE010E000A04E100000001F3D71D
:103720000301640E366F0001E4DED5D739D083AED5
:1037300037D0C80EF66E080EF76E196AF2BE198EF3
:10374000F29EA8EC03F019BEF28E3750020828E171
:1037500083AE26D0BF07BF53D8B4BF6B120E030190
:10376000876F886B400E896F8A6B8B6BBFC08CF341
:103770008D6B8E6B000188EC09F0DAEC09F001C06A
:1037800035F3000E030101BE010E000A04E1000042
:103790000001F3D70301640E366F0001AADED8D70B
:1037A0000AEF27F0B60E006E036A026A016A03018F
:1037B0003B513C113D113E1102E1006A0DD0D89001
:1037C00001BE09D03B373C373D373E370336023622
:1037D0000136002EF4D7019E0001000C0301436B5B
:1037E000446B010E456FDA6AD96A030E486F3B0ECF
:1037F000476F030EEA6E3F0EE96E48C3E2FF47C310
:10380000E1FF45C346F3D890E550EE02F350432361
:10381000F4504423462FF7D743C3DEFF44C343F39A
:10382000446BD8B0442B472BD8B4482B452B45517B
:103830000508DFE10001CEEF1FF0030142514419FA
:10384000800B466F42AF05D0411F421F412BD8B4B9
:10385000422B44AF05D0431F441F432BD8B4442B05
:10386000016A026A006A036A445102E1435118E0A6
:10387000100E456FD8904137423700360336445119
:10388000035C02E14351005C07E34351005ED8A0B2
:1038900003064451035ED88001360236452FEAD72D
:1038A00046AF05D0011E021E012AD8B4022A00012B
:1038B0008EEF1CF0030142514419800B466F42AF5A
:1038C00005D0411F421F412BD8B4422B44AF05D035
:1038D000431F441F432BD8B4442B41514303F3CF20
:1038E00001F0F4CF00F04403F350002642514303AB
:1038F000F3500020026E46AF05D0011E021E012AC1
:10390000D8B4022A00019BEF1CF03AC342F339C33A
:1039100041F33CC344F33BC343F38FD702C03EF3B0
:1039200001C03DF33CC342F33BC341F33EC344F308
:103930003DC343F3BFD701500301395D3F6F0250D0
:103940003A59406F3DC300F03EC301F03FC302F05F
:1039500040C303F0000107EF20F0EACF3FF3E9CFC7
:103960003EF303013839F0093A6F3A27E20F3B6F13
:10397000320F3D6F38510F0B3B273B273D27E90F97
:103980003C6F3C273C2737390F0B3C273D273C3702
:103990003D373D1F3D3737510F0B3D273A37070E57
:1039A000396F0A0E3C073D27FDE33B073C27FDE34B
:1039B0003A073B27FDE339073A27FDE3030EEA6E9A
:1039C000390EE96E070E3E153E9DE9263D0EE95C77
:1039D000D8B43E8DEF50006E08E13EBD06D03EB932
:1039E0000CD03EB702D0200E03D03E873E99300E59
:1039F000002600509EA8FED7AD6EEE503EADE6D735
:103A00000001000CE1C0EAF0E0C0E9F0EA3903018E
:103A1000376F0F0E371737510F0B3F6EECC0EEF0BC
:103A2000EBC0EDF0EAC0ECF0E9C0EBF00001ED51C5
:103A3000EB5D03E1EE51EC5D13E0EB51E95D03E179
:103A4000EC51EA5D0DE0E95302E1EA5309E0EF6B66
:103A5000140E0201FF6F0001F06BF16B8DEF24F08B
:103A6000E3310301386F0001E2310301376F38336E
:103A70003733383337333833373338333733070E48
:103A8000381737511F0B0001EF6FE3C037F3030105
:103A90003751F00B0001F46F0301376B0001E35164
:103AA000080B0301386F375307E13851080804E168
:103AB0000B0E0001F41303D00A0E0001F413F451AD
:103AC0004A08D8A413EF22F003012A6BD890000112
:103AD000E531036EE4310301026F03C003F3046BAD
:103AE000056B0001E251010B0301376F386B372D75
:103AF00007D0385305E1800E0327000E0423052369
:103B00000001E251020B0301376F386B3751020895
:103B100006E1385304E1010E0427000E052326A810
:103B20001DD0780EF66E060EF76E080E806F00013F
:103B30009AEC04F0410EE96E05C37CF304C37BF3F9
:103B400003C37AF302C379F32EEC16F00A0E9EA893
:103B5000FED7AD6E0D0E9EA8FED7AD6E0001E451EE
:103B6000010B0301376F386B3735026E3835036E42
:103B7000023603360236033602360336F00E0216DC
:103B800002C027F30001E7390301376F386B0F0ECE
:103B9000371737510F0B006E036A0050386B27C37D
:103BA00037F327BF38072725016E3851032201C09C
:103BB00027F30001E7310301386F0001E63103010B
:103BC000376F383337333833373338333733383365
:103BD000373338333733030E381737513F0B286FDD
:103BE000296B0001E6AB03D00301292B0001E6514C
:103BF0000F0B0301266F29530BE1D890263127279D
:103C000027BF05D02751170802E2180E275F07D0FB
:103C1000D8902631275F27AF02D0180E272705C37B
:103C20003EF304C33DF303C33CF302C33BF3000183
:103C3000B9DD00C037F301C038F302C039F303C067
:103C40003AF3D88203C094F302C093F301C092F315
:103C500000C091F3CD0E0301986F980E976F6B0E15
:103C6000966F8C0E956F000191EC0AF000C037F34F
:103C700001C038F302C039F303C03AF303C08BF339
:103C800002C08AF301C089F300C088F303018F6B7F
:103C9000A00E8E6F360E8D6F870E8C6F0001CDECEF
:103CA0000BF003C094F302C093F301C092F300C081
:103CB00091F3D3EC0FF003C009F302C008F301C085
:103CC00007F300C006F305C33EF304C33DF303C38B
:103CD0003CF302C33BF366DD00C037F301C038F3A9
:103CE00002C039F303C03AF3D88203C094F302C090
:103CF00093F301C092F300C091F3660E0301986F35
:103D0000B00E976F690E966F8C0E956F000191EC57
:103D10000AF000C037F301C038F302C039F303C022
:103D20003AF309C33EF308C33DF307C33CF306C3AC
:103D30003BF338DD00C03BF301C03CF302C03DF370
:103D400003C03EF303C094F302C093F301C092F3A7
:103D500000C091F30301986BA00E976F360E966F1B
:103D6000870E956F000116EC0AF003C094F302C0B1
:103D700093F301C092F300C091F3D3EC0FF003C0B2
:103D80003EF302C03DF301C03CF300C03BF30ADD4B
:103D9000D8823AC394F339C393F338C392F337C349
:103DA00091F303C098F302C097F301C096F300C0EB
:103DB00095F391EC0AF000C037F301C038F302C06C
:103DC00039F303C03AF303C08BF302C08AF301C096
:103DD00089F300C088F3010E03018F6FCD0E8E6F43
:103DE000740E8D6F830E8C6F0001CDEC0BF003C051
:103DF00094F302C093F301C092F300C091F3D3ECAB
:103E00000FF003C015F302C014F301C013F300C098
:103E100012F36C0E0301025D376F3A0E0359386FCF
:103E2000000E0459396F000E05593A6F09C33EF36D
:103E300008C33DF307C33CF306C33BF30001B2DC08
:103E400000C03BF301C03CF302C03DF303C03EF3AE
:103E500003C094F302C093F301C092F300C091F346
:103E60000301986BA00E976F360E966F870E956FB5
:103E7000000116EC0AF003C094F302C093F301C0F2
:103E800092F300C091F3D3EC0FF000500301375FC1
:103E90000150385B0250395B03503A5B15C33EF367
:103EA00014C33DF313C33CF312C33BF300017ADCAC
:103EB00000C03BF301C03CF302C03DF303C03EF33E
:103EC00003C094F302C093F301C092F300C091F3D6
:103ED000010E0301986FCD0E976F740E966F830ECF
:103EE000956F000116EC0AF003C094F302C093F33F
:103EF00001C092F300C091F3D3EC0FF00050030126
:103F0000375D166F01503859176F02503959186FC5
:103F100003503A59196F12510E0806E1135304E188
:103F2000145302E1155309E012510F080CE1135329
:103F30000AE1145308E1155306E11D6B1C6B1B6B62
:103F4000010E1A6F04D01D6B1C6B1B6B1A6B1A5180
:103F500006250A6F1B5107210B6F1C5108210C6F9E
:103F60001D5109210D6F010E125D376F000E13599F
:103F7000386F000E1459396F000E15593A6F1DC372
:103F80003EF31CC33DF31BC33CF31AC33BF3426B2C
:103F9000416B406B0C0E3F6F000120D400500301B9
:103FA000375D1E6F015038591F6F02503959206F0D
:103FB00003503A59216F6C0E0A27070E0B23000E8F
:103FC0000C230D23020E0225376F000E0321386FDC
:103FD000000E0421396F000E05213A6F350E375D52
:103FE0000E6FD10E38590F6F000E3959106F000E39
:103FF0003A59116F0FC338F30EC337F30FC33AF3B7
:104000000EC339F33C6B070E3B6F00017ED403C037
:1040100036F302C035F301C034F300C033F3010EB0
:1040200003013525016E000E3621036E01C000F03C
:10403000026A036A03C025F302C024F3236F00C0A1
:1040400022F3222D16D0235314E1245312E12553D9
:1040500010E1030EEA6E2B0EE96E000E000101EC7A
:1040600002F00A000900F550EE6E0009FBE195D060
:1040700003012251020816E1235314E1245312E1F3
:10408000255310E1030EEA6E2B0EE96E000E0001BF
:104090000BEC02F00A000900F550EE6E0009FBE19E
:1040A0007CD003012251030816E1235314E1245369
:1040B00012E1255310E1030EEA6E2B0EE96E000E9D
:1040C000000115EC02F00A000900F550EE6E00093F
:1040D000FBE163D003012251040816E1235314E1EC
:1040E000245312E1255310E1030EEA6E2B0EE96E04
:1040F000000E00011FEC02F00A000900F550EE6E00
:104100000009FBE14AD003012251050816E12353BF
:1041100014E1245312E1255310E1030EEA6E2B0E35
:10412000E96E000E000129EC02F00A000900F550CA
:10413000EE6E0009FBE131D003012251060816E1C1
:10414000235314E1245312E1255310E1030EEA6EC8
:104150002B0EE96E000E000133EC02F00A0009009C
:10416000F550EE6E0009FBE118D00301225107085B
:1041700015E1235313E1245311E125530FE1030EFD
:10418000EA6E2B0EE96E000E00013DEC02F00A0013
:104190000900F550EE6E0009FBE103011E2D16D05B
:1041A0001F5314E1205312E1215310E1030EEA6E74
:1041B0002F0EE96E000E000147EC02F00A00090024
:1041C000F550EE6E0009FBE112D103011E51020809
:1041D00016E11F5314E1205312E1215310E1030EA5
:1041E000EA6E2F0EE96E000E000151EC02F00A009B
:1041F0000900F550EE6E0009FBE1F9D003011E51F4
:10420000030816E11F5314E1205312E1215310E17A
:10421000030EEA6E2F0EE96E000E00015BEC02F059
:104220000A000900F550EE6E0009FBE1E0D0030141
:104230001E51040816E11F5314E1205312E12153CB
:1042400010E1030EEA6E2F0EE96E000E000165EC20
:1042500002F00A000900F550EE6E0009FBE1C7D03C
:1042600003011E51050816E11F5314E1205312E10A
:10427000215310E1030EEA6E2F0EE96E000E0001CD
:104280006FEC02F00A000900F550EE6E0009FBE148
:10429000AED003011E51060816E11F5314E120534E
:1042A00012E1215310E1030EEA6E2F0EE96E000EAB
:1042B000000179EC02F00A000900F550EE6E0009E9
:1042C000FBE195D003011E51070816E11F5314E1CD
:1042D000205312E1215310E1030EEA6E2F0EE96E16
:1042E000000E000183EC02F00A000900F550EE6EAA
:1042F0000009FBE17CD003011E51080816E11F53A1
:1043000014E1205312E1215310E1030EEA6E2F0E47
:10431000E96E000E00018DEC02F00A000900F55074
:10432000EE6E0009FBE163D003011E51090816E19E
:104330001F5314E1205312E1215310E1030EEA6EE2
:104340002F0EE96E000E000197EC02F00A00090042
:10435000F550EE6E0009FBE14AD003011E510A0838
:1043600016E11F5314E1205312E1215310E1030E13
:10437000EA6E2F0EE96E000E0001A1EC02F00A00B9
:104380000900F550EE6E0009FBE131D003011E512A
:104390000B0816E11F5314E1205312E1215310E1E1
:1043A000030EEA6E2F0EE96E000E0001ABEC02F078
:1043B0000A000900F550EE6E0009FBE118D0030178
:1043C0001E510C0815E11F5313E1205311E1215335
:1043D0000FE1030EEA6E2F0EE96E000E0001B5EC40
:1043E00002F00A000900F550EE6E0009FBE103013E
:1043F0000D530AE10C5308E10B51060812E2FF0AC3
:1044000003E10A51D9080DE20D530BE10C5309E108
:104410000B51070806E303E10A51E90802E3010E24
:104420002A6F7CD20001F4510A0803E0F4510B0812
:1044300067E1000E26B8010E01081FE2F4510A08D8
:104440000DE1300E9EA8FED7AD6E410E9EA8FED7A0
:10445000AD6E200E9EA8FED7AD6E0FD0F4510B08A6
:104460000CE1300E9EA8FED7AD6E420E9EA8FED780
:10447000AD6E200E9EA8FED7AD6EE251030B030178
:10448000376F386BD8903735026E383502C0F5F08B
:104490000001010EF525036AF60FE96E000E0320F8
:1044A000EA6EE6C0EFFF036AF551F60FE96E000E03
:1044B0000320EA6E0301E7C0EFFF0001F06BF16B30
:1044C0000301376B0001E351040B0301386F3753CD
:1044D00006E13851040803E1010E0001F06F00010C
:1044E000E251100B0301376F386B3751100806E1AA
:1044F000385304E1010E0001F16F03010FD20001F6
:10450000F4512A08D8A481D0E251100B0301376F6F
:10451000386B3751100806E1385304E1010E0101F0
:10452000006F02D00101006B0001E2510F0B03018B
:10453000376F386B3735026E3835036E0236033607
:10454000FC0E021602C0FFF00001010100532DE134
:10455000030E0001FF25036A010FE96E010E03201F
:10456000EA6EE6C0EFFF020EFF25036A010FE96E57
:10457000010E0320EA6E0301E7C0EFFF010E000108
:10458000FF25036A010FE96E010E0320EA6EE4C005
:10459000EFFF036AFF51010FE96E010E0320EA6E7F
:1045A0000301E5C0EFFF2ED00101002D2CD0030E3A
:1045B0000001FF25036A830FE96E010E0320EA6EF6
:1045C000E6C0EFFF020EFF25036A830FE96E010EBE
:1045D0000320EA6E0301E7C0EFFF010E0001FF2593
:1045E000036A830FE96E010E0320EA6EE4C0EFFF59
:1045F000036AFF51830FE96E010E0320EA6E030187
:10460000E5C0EFFF01018BD10001F4513A08D8A4B5
:1046100089D0E5AF01D081D1E5BD4AD0E5310301B4
:10462000386F0001E4310301376F383337333833E3
:104630003733383337333833373338333733030E80
:10464000381737513F0B406E442C30D0860EF66E33
:10465000060EF76E080E806F00019AEC04F03FC062
:1046600079F3570E03017A6F00010BEC16F0900EF0
:10467000F66E060EF76E050E0301806F00019AECD0
:1046800004F040C079F3570E03017A6F00010BEC80
:1046900016F0200E9EA8FED7AD6E0A0E9EA8FED77D
:1046A000AD6E0D0E9EA8FED7AD6E030139D0000190
:1046B000E5AD35D0E5310301386F0001E431030188
:1046C000376F38333733383337333833373338335A
:1046D000373338333733030E381737513F0B416EBA
:1046E000442C1ED09C0EF66E060EF76E090E806FDF
:1046F00000019AEC04F041C079F3570E03017A6F80
:1047000000010BEC16F0200E9EA8FED7AD6E0A0E2F
:104710009EA8FED7AD6E0D0E9EA8FED7AD6E03010E
:10472000FDD00001F4518A08D8A4F7D0010EF26F31
:10473000E3C039F0E2C038F0E5C03BF0E4C03AF045
:10474000E7C03DF0E6C03CF0269238B826822694B9
:1047500038B626843850070B3E6E0301376B3B504A
:10476000400B386F375305E13851400802E126808D
:1047700001D02690376B3B50800B386F375305E1E3
:104780003851800802E1268601D026963AC028F0EA
:104790003B50070B296E3B30376F373337331F0ED3
:1047A00037173751070B276E3DC025F03CC024F06A
:1047B000442C44D0000E26B2010E376F000E26B4F2
:1047C000010E386FAC0EF66E060EF76E070E806F98
:1047D00000019AEC04F037C380F31B0E0301816FD4
:1047E0000001C5EC04F0200E9EA8FED7AD6E460E6B
:1047F0009EA8FED7AD6E3D0E9EA8FED7AD6E38C307
:1048000080F31B0E0301816F0001C5EC04F0BA0EAA
:10481000F66E060EF76E040E0301806F00019AEC2F
:1048200004F03EC080F31B0E0301816F0001C5EC54
:1048300004F0200E9EA8FED7AD6E0301442C40D09C
:10484000000E26B6010E376F000E26B0010E386F2F
:10485000440E9EA8FED7AD6E3D0E9EA8FED7AD6E4F
:1048600037C380F31B0E816F0001C5EC04F0C60E48
:10487000F66E060EF76E050E0301806F00019AECCE
:1048800004F038C380F31B0E0301816F0001C5ECF7
:1048900004F0CD0EF66E060EF76E050E0301806F66
:1048A00000019AEC04F027C080F31B0E0301816F16
:1048B0000001C5EC04F0200E9EA8FED7AD6E0301EA
:1048C000442C2CD0D60EF66E060EF76E040E806FBA
:1048D00000019AEC04F0100EE96E29C038F328C0EC
:1048E00037F3ADEC1CF0DD0EF66E060EF76E050E1E
:1048F0000301806F00019AEC04F0100EE96E25C0F0
:1049000038F324C037F3ADEC1CF00A0E9EA8FED796
:10491000AD6E0D0E9EA8FED7AD6E03010101000124
:10492000E9EF24F0240E0301876F886B896B8A6B93
:104930008B6B8C6B8D6B8E6B000188EC09F053ECEC
:104940000FF001C033F3000E030133BF010E000A64
:1049500006E1350E006E002EFED70001F0D70001F3
:10496000C151010B01E135D0C251010B01E131D040
:10497000C3C0E8F0E16BC4C0E0F0E0C0E1F0E06B80
:10498000C551E027000EE123E05303E1E15301E1CB
:1049900020D0E36BC6C0E2F0E2C0E3F0E26BC751A7
:1049A000E227000EE323E56BC8C0E4F0E4C0E5F0C5
:1049B000E46BC951E427000EE523E76BCAC0E6F0BB
:1049C000E6C0E7F0E66BCB51E627000EE72302EFE7
:1049D0001DF019EF27F0EF5210E0EACF34F3E9CFE2
:1049E00033F3EFCF91F3C5EC08F034C3EAFF33C3E0
:1049F000E9FFE92AD8B4EA2AEED7000C030134BF54
:104A000012D00F0E006E333900160A0E005C03E25E
:104A1000300E002602D03451002600C091F3000170
:104A2000C5EC08F003010F0E33170A0E335D02E2E6
:104A3000300E02D0349F3451332733C391F3000139
:104A4000C5EC08F0000CE9500301376F3B0E3E6FD8
:104A50009A0E3D6FCA0E3C6F3B6B0A0E396FD882BF
:104A6000030EEA6E330EE96E36C394F335C393F347
:104A700034C392F333C391F33EC398F33DC397F32A
:104A80003CC396F33BC395F30001F4EC0FF00150E7
:104A9000005213E103013951010AD8A402D00001E8
:104AA0000CD037510CE00F0B395D01E010E237BF3D
:104AB0000ED037BD04D0200E03D00301376B300E6B
:104AC000002600C091F30001C5EC08F00301D89264
:104AD0003EC394F33DC393F33CC392F33BC391F3C2
:104AE000986B976B966B0A0E956F0001F4EC0FF0C4
:104AF00003C03EF302C03DF301C03CF300C03BF3F2
:104B00000301392FACD70001FBEF27F0F86AD09EE4
:104B1000078E5E0E006E100E016E020EE96E000E24
:104B2000EA6EEE6A002EFDD7012EFBD7EA6AE96A2B
:104B3000700ED36E400E9B6ED350B8868A0EAF6E49
:104B4000000EB06EA60EAC6E900EAB6E566A576A33
:104B5000000E7E6EC198C19A7F50E00B7F6E799AED
:104B600079987A6A7B6A1A6A1B6A700ED36ED35080
:104B7000C290000E7E6EC198C19A7F50E00B7F6E8E
:104B80000F0E926E0B0E936E800E946ED10E956E7C
:104B90009690968296849686D1907C92C00EF21260
:104BA0009D8A0F0EAC6FFF0EAD6F8B8A949A899E13
:104BB000929E080EF66E080EF76E196AF2BE198EF6
:104BC000F29EA8EC03F019BEF28E0E0EF66E080EE1
:104BD000F76E196AF2BE198EF29EA8EC03F019BEA8
:104BE000F28EF2CF33F3F29EAA6A0A0EA96EA69C49
:104BF000A69EA680A850030133BFF28E0001A06FCD
:104C00004A0EF66E080EF76E060E0301806F000165
:104C10009AEC04F0A0C080F31B0E0301816F000129
:104C2000C5EC04F00A0E9EA8FED7AD6E0D0E9EA830
:104C3000FED7AD6EA03D19D0020EA06FAA6A0A0E73
:104C4000A96E020EA86EA69CA69EA684F250006EC7
:104C5000F29E0F01550EA76EAA0EA76EA682A6B2EF
:104C6000FED7A6940050F212000183AC1AD0010EB8
:104C7000A06FAA6A0A0EA96EA0C0A8FFA69CA69E55
:104C8000A684F250006EF29E0F01550EA76EAA0E7A
:104C9000A76EA682A6B2FED7A6940050F21239D013
:104CA0000001928280A21AD0020EA06FAA6A0A0E98
:104CB000A96EA0C0A8FFA69CA69EA684F250006E76
:104CC000F29E0F01550EA76EAA0EA76EA682A6B27F
:104CD000FED7A6940050F2121CD00001928080A052
:104CE00019D0030EA06FAA6A0A0EA96EA0C0A8FF71
:104CF000A69CA69EA684F250006EF29E0F01550E51
:104D0000A76EAA0EA76EA682A6B2FED7A6940050E2
:104D1000F212000183AC01D0FDD7928280A201D0B3
:104D2000FCD7928080A001D0FCD7560EF66E080EFC
:104D3000F76E060E0301806F00019AEC04F0A0C02C
:104D400080F31B0E0301816F0001C5EC04F00A0E15
:104D50009EA8FED7AD6E0D0E9EA8FED7AD6E26881E
:104D600026EF05F00FEF06F00301846B200E856F30
:104D7000000147EC06F0010EBD6FBC6FBB6BBA6B58
:104D80000F0EB96FFF0EB86F620EF66E080EF76E5B
:104D9000060E0301336F000101EF09F0A0C037F3E5
:104DA0001B0E0301386F000116EC09F0060E03011B
:104DB000846F300E856F000147EC06F0020EBD6F68
:104DC000BC6F0F0EBB6FBA6BB96FFF0EB86F6C0E76
:104DD000F66E080EF76E56EC09F0010EBD6FBC6F53
:104DE000CFEF0DF038EC11F06CEC12F0020E376ED4
:104DF000010E446E010EA327D8B0A42BD8B4A52B66
:104E0000D8B4A62B5750565C03E0CEEF17F0FAD774
:104E10008EEF1AF0DAEC09F001C033F3000E030153
:104E200001B4010E010805E13750030802E000015A
:104E300079D50001A6530EE1A5530CE1A4510E084B
:104E4000D8B096EF2BF0FF0A05E1A3519F08D8B028
:104E500096EF2BF038EC11F08EEC16F0240E0301D7
:104E6000846F100E856F000147EC06F0BB6BBA6BC8
:104E70000F0EB96FFF0EB86FF22D07D08E0EF66EC3
:104E8000050EF76E56EC09F018D0F02D10D0F12D6C
:104E900007D0740EF66E080EF76E56EC09F006D0C9
:104EA000780EF66E080EF76E56EC09F006D07C0E02
:104EB000F66E080EF76E56EC09F0020EBC6FBD6F71
:104EC0000301846B856B000147EC06F00C0EBB6F91
:104ED000BA6B0F0EB96FFF0EB86FEA6AF60EE96E85
:104EE0007ADD010EBC6FBD6F390E0301846F100EA9
:104EF000856F000147EC06F0BB6BBA6B0F0EB96F04
:104F0000FF0EB86FEAC033F3570E0301346F000190
:104F100075DDE9C033F3570E0301346F00016EDD18
:104F200003012A2D6AD026BA68D0846B180E856FCB
:104F3000000147EC06F0BB6BBA6B040EB96FF40EC0
:104F4000B86F0301366B356B346B27C333F327C35C
:104F500037F3110E386F000116EC09F03A0E030119
:104F6000916F0001C5EC08F00301366B356B346BB3
:104F700028C333F328C337F3010E386F000116EC52
:104F800009F0200E0301916F0001C5EC08F0220E1C
:104F90000301846F180E856F000147EC06F0030EC5
:104FA000EA6E2F0EE96E17DD200E0301916F0001EE
:104FB000C5EC08F0360E0301846F180E856F0001F2
:104FC00047EC06F016C337F3110E0301386F0001EA
:104FD00016EC09F02C0E0301916F0001C5EC08F0EE
:104FE000040EE96E0DC336F30CC335F30BC334F373
:104FF0000AC333F328D503012A6B0001F25304E0FE
:105000004552D8A492EF2BF0010E03017A6F796F0D
:105010000001A8EC13F0015002080DE3010E03019A
:105020007A6F830E796F0001A8EC13F0015002082B
:1050300002E38CEF2BF0A753D8A4B6D1A853D8A481
:10504000B3D1A953D8A4B0D1AA53D8A4ADD1536A2F
:10505000526A5250400802E1535225E0010E522498
:10506000E96E010E5320EA6EEF50F00B18E153C0C9
:1050700055F052C054F05450400802E155520CE033
:10508000010E5424E96E010E5520EA6E200EEF6EDB
:10509000542AD8B4552AEFD70101416B0001522A96
:1050A000D8B4532AD6D70201056B416B7D6BB96B1F
:1050B00001010151200801E170D10001BB6BBA6B05
:1050C0000F0EB96FF20EB86F4F6A100E4E6E4E5241
:1050D00002E14F5222E0010E4E24E96E010E4F20F4
:1050E000EA6EEF50200814E1020E03017B6F050EFB
:1050F0007A6F010E7D6F7C6F4FC07FF34EC07EF3E1
:10510000000104EC15F04FC047F04EC046F005D04A
:105110004E50D8B44F064E06DAD747C051F046C0BD
:1051200050F05050100802E151520CE0050E50248E
:10513000E96E020E5120EA6E200EEF6E502AD8B4AE
:10514000512AEFD70201156B0301846B200E856F86
:10515000000147EC06F0020EEA6E050EE96E3BDC3C
:10516000100E46244E6E000E47204F6E46504E5C89
:1051700003E147504F5C2DE0010E4E24E96E010E15
:105180004F20EA6EEF5020081FE1010E4624030174
:10519000336F010E4720346F010E3327000E342386
:1051A000020E7B6F410E7A6F34C37DF333C37CF301
:1051B0004FC07FF34EC07EF3000104EC15F04FC0EA
:1051C00049F04EC048F005D04E50D8B44F064E06B8
:1051D000CDD74650485C506E47504958516E50509C
:1051E000100802E151520CE0410E5024E96E020E0B
:1051F0005120EA6E200EEF6E502AD8B4512AEFD714
:105200000201516B0301846B280E856F000147EC8E
:1052100006F0020EEA6E410EE96EEBEC24F0100E81
:1052200048244E6E000E49204F6E48504E5C03E1FC
:1052300049504F5C2DE0010E4E24E96E010E4F20C7
:10524000EA6EEF5020081FE1010E48240301336F7E
:10525000010E4920346F010E3327000E3423020E55
:105260007B6F7D0E7A6F34C37DF333C37CF34FC005
:105270007FF34EC07EF3000104EC15F04FC04BF0FD
:105280004EC04AF005D04E50D8B44F064E06CDD78A
:1052900048504A5C506E49504B58516E505010085F
:1052A00002E151520CE07D0E5024E96E020E5120B5
:1052B000EA6E200EEF6E502AD8B4512AEFD70201C1
:1052C0008D6B0301846B300E856F000147EC06F097
:1052D000020EEA6E7D0EE96EEBEC24F0100E4A240D
:1052E0004E6E000E4B204F6E4A504E5C03E14B5009
:1052F0004F5C2DE0010E4E24E96E010E4F20EA6E48
:10530000EF5020081FE1010E4A240301336F010E04
:105310004B20346F010E3327000E3423020E7B6FB7
:10532000B90E7A6F34C37DF333C37CF34FC07FF380
:105330004EC07EF3000104EC15F04FC04DF04EC09E
:105340004CF005D04E50D8B44F064E06CDD74A503B
:105350004C5C506E4B504D58516E5050100802E14D
:1053600051520CE0B90E5024E96E020E5120EA6E43
:10537000200EEF6E502AD8B4512AEFD70201C96B24
:105380000301846B380E856F000147EC06F0020EB6
:10539000EA6EB90EE96EEBEC24F00001AA6BA96B82
:1053A000A86B010EA76FB8D1A72DB6D1A853D8A46A
:1053B000B3D1A953D8A4B0D1AA53D8A4ADD1536ABC
:1053C000526A5250400802E1535225E0830E5224A3
:1053D000E96E010E5320EA6EEF50F00B18E153C056
:1053E00055F052C054F05450400802E155520CE0C0
:1053F000830E5424E96E010E5520EA6E200EEF6EE6
:10540000542AD8B4552AEFD70101C36B0001522AA0
:10541000D8B4532AD6D70201236B5F6B9B6BD76B33
:1054200001018351200801E172D10001BB6BBA6B0D
:10543000040EB96F4F0EB86F4F6A100E4E6E4E527B
:1054400002E14F5223E0830E4E24E96E010E4F20FD
:10545000EA6EEF50200815E1020E03017B6F230E68
:105460007A6F010E7D6F830E7C6F4FC07FF34EC04D
:105470007EF3000104EC15F04FC047F04EC046F03B
:1054800005D04E50D8B44F064E06D9D747C051F07C
:1054900046C050F05050100802E151520CE0230E6B
:1054A0005024E96E020E5120EA6E200EEF6E502A53
:1054B000D8B4512AEFD70201336B0301846B200E5D
:1054C000856F000147EC06F0020EEA6E230EE96ECE
:1054D000EBEC24F0100E46244E6E000E47204F6E6B
:1054E00046504E5C03E147504F5C2DE0830E4E2446
:1054F000E96E010E4F20EA6EEF5020081FE1830E87
:1055000046240301336F010E4720346F010E332709
:10551000000E3423020E7B6F5F0E7A6F34C37DF36F
:1055200033C37CF34FC07FF34EC07EF3000104EC25
:1055300015F04FC049F04EC048F005D04E50D8B4D9
:105540004F064E06CDD74650485C506E47504958DE
:10555000516E5050100802E151520CE05F0E502481
:10556000E96E020E5120EA6E200EEF6E502AD8B47A
:10557000512AEFD702016F6B0301846B280E856FF0
:10558000000147EC06F0020EEA6E5F0EE96EEBECEE
:1055900024F0100E48244E6E000E49204F6E4850E5
:1055A0004E5C03E149504F5C2DE0830E4E24E96EC2
:1055B000010E4F20EA6EEF5020081FE1830E4824B1
:1055C0000301336F010E4920346F010E3327000EA3
:1055D0003423020E7B6F9B0E7A6F34C37DF333C38B
:1055E0007CF34FC07FF34EC07EF3000104EC15F056
:1055F0004FC04BF04EC04AF005D04E50D8B44F06C5
:105600004E06CDD748504A5C506E49504B58516EAB
:105610005050100802E151520CE09B0E5024E96EEC
:10562000020E5120EA6E200EEF6E502AD8B4512A95
:10563000EFD70201AB6B0301846B300E856F000165
:1056400047EC06F0020EEA6E9B0EE96EEBEC24F0DE
:10565000100E4A244E6E000E4B204F6E4A504E5C88
:1056600003E14B504F5C2DE0830E4E24E96E010E9A
:105670004F20EA6EEF5020081FE1830E4A240301F9
:10568000336F010E4B20346F010E3327000E34238D
:10569000020E7B6FD70E7A6F34C37DF333C37CF376
:1056A0004FC07FF34EC07EF3000104EC15F04FC0F5
:1056B0004DF04EC04CF005D04E50D8B44F064E06BB
:1056C000CDD74A504C5C506E4B504D58516E505097
:1056D000100802E151520CE0D70E5024E96E020E80
:1056E0005120EA6E200EEF6E502AD8B4512AEFD71F
:1056F0000201E76B0301846B380E856F000147ECF4
:1057000006F0020EEA6ED70EE96EEBEC24F0000113
:10571000AA6BA96BA86BA76BBB6BBA6B0F0EB96FAB
:10572000FF0EB86FA66BA56BA46BA36BFAEF26F008
:02573000030074
:020000040030CA
:0E00000000C8181E008F80000FC00FE00F40D8
:00000001FF
